:020000020000FC
:0200000012C02C
:02000600A8C28E
:100026000FE50DBF04E00EBFA89500E004BF08E190
:1000360001BD00E101BD0FE307BB0EEF01BB02E20C
:1000460004BBA99AAD9AC59A929A949A08E10AB9FC
:1000560006E800BD00E000BD0CE009B908E103BDFB
:100066000AE005BD00E809BF78948BD243504D20C5
:100076006F6E20616E204156522C2076312E300D47
:1000860000007FD2496E6974696E67206D6D632EBC
:100096002E2E0D0024D150E060E00BEC23D201E0BF
:1000A60010E0500F611FC8F760E050E067D1E0E64E
:1000B600F0E060E250E00191FF93EF9313D2EF91ED
:1000C600FF9101E010E0500F611FE03EA1F7F03014
:1000D60091F700E0802F00E2902F20E052D20D4FE2
:1000E6006B2C20435055206973206C697665210D71
:1000F600000020E0913018F09C3D08F421E0582FD4
:10010600692FC9D1019610E0E0E7FAE0E00FF11F90
:10011600E00FF11F7591A491072F0F71003059F070
:1001260010E0000FE2ECF5E0E00FF11F05911491ED
:10013600E02FF12F09950A2F0C7F0695003051F01C
:10014600E4E6F7E010E0E00FF11F05911491E02FCF
:10015600F12F09957295A295072F0E70A0730A2BA1
:10016600003051F0E6E9F6E010E0E00FF11F0591EE
:100176001491E02FF12F0995BCCF103091F011307A
:10018600A1F00895103099F01230D1F01031D1F06D
:100196001231D1F01431D1F01531D1F01631D1F040
:1001A600089500E05F990FEF089500D20895E9D110
:1001B60044656275673A2000DFD1E3D10D000895EA
:1001C600F9D10895B02E0895C02E0895E02E089511
:1001D600D02E08950F935C2D60E01B2D103031F06A
:1001E6000AE1500F00E0601F1A95F8CF0F91013019
:1001F60011F0023019F15F936695579566955795FC
:10020600BDD05F91E0E6F0E000E810E050FDE00FC1
:1002160050FDF11F51FDF3956D2D5E2D10E81F93D6
:100226000191FF93EF935ED1EF91FF9101E010E012
:10023600500F611F1F911A9591F708955F936F9361
:10024600669557956695579599D06F915F915F938F
:100256006F93E0E6F0E000E810E050FDE00F50FD9F
:10026600F11F51FDF3956D2D5E2D10E81F93FF9341
:10027600EF9311D1EF91FF91019301E010E0500F40
:10028600611F1F911A9591F76F915F91669557952A
:10029600669557959BD008950FEF0FB90EB107FFDE
:1002A600FDCF0FB10895E0E0F0E0F6DF0F3F21F457
:1002B6003196FF3F11F0F9CF0895012F5DD161D13D
:1002C6003A204572726F723A204D4D432072657323
:1002D600702074696D656F7574210D00A3C003E508
:1002E6000DB9949A14E1012FD8DF1A95E1F7949885
:1002F600D3DFD2DFD1DFD0DFCFDFCEDF949ACCDF02
:10030600CBDFCADFC9DF94980FEFC7DF0FEFC5DF7A
:1003160000E4C3DF00E0C1DF00E0BFDF00E0BDDFD7
:1003260000E0BBDF05E9B9DF0FEFB7DF10E0BBDFA9
:10033600949AB2DF16E91F9394980FEFAEDF01E4AB
:10034600ACDF00E0AADF00E0A8DF00E0A6DF00E007
:10035600A4DF05E9A2DFA0DF11E0A5DF003041F050
:10036600949A9ADF1F911A95103029F704E0A5CFC9
:100376001F91949A91DF00E00DB9089500E50DB93B
:1003860094988ADF01E589DF00E0550F661F001F9C
:1003960084DF062F82DF052F80DF00E07EDF05E9A0
:1003A6007CDF0FEF7ADF12E07EDF13E07CDFE0E632
:1003B600F0E072DF0193E036E1F7F230D1F76CDF5F
:1003C6006BDF949A69DF00E00DB9089500E50DB979
:1003D600949862DF08E561DF00E0550F661F001F95
:1003E6005CDF062F5ADF052F58DF00E056DF05E9F0
:1003F60054DF0FEF52DF11E056DF0EEF4EDFE0E67F
:10040600F0E001914ADFE036E1F7F230D1F744DF60
:1004160043DF42DF41DF0F3FE9F7949A3DDF00E01B
:100426000DB90895F89400E101BD0EE701BDFFCFB7
:100436000F9302B3077102BB08B3007E08BBE0FD51
:10044600C49AE1FDC39AE2FDC29AE3FDC19AE4FDB6
:10045600C09AE5FD959AE6FD969AE7FD979AF0FD16
:10046600939A0F910895007F989901609A99026076
:100476009C9904609B99086008951F9315B3127E9A
:1004860000FD116001FD146002FD106103FD18609E
:1004960015BB1F910895F894E62FF0E0152F110F64
:1004A600EE1FFF1FC5DFC598F0E0E52FEF77C0DF31
:1004B6000000AD980000000092980000D4DF929AE8
:1004C6000295AD9AF0E0E52FE068B2DF0000AD9846
:1004D6000000929800000000C6DF929AAD9AC59A75
:1004E60078940895F89414B31D6114BBC6DFE62F03
:1004F600F0E0152F110FEE1FFF1F9ADF000000001E
:10050600C598F0E0E52FE06893DF00000000AD98A5
:1005160000000000A998000000000000A99AAD9A0A
:10052600F0E0E52FEF7784DF0295A7DFAD980000B6
:100536000000A99800000000A99A00000000AD9AEA
:10054600C59A04B3027E04BB05B3027E05BB78944C
:1005560008950000AD98C5980000AD9AC59A189503
:100566000F930F700A3020F0095C24D00F91089584
:10057600005D20D00F9108950295F2DF0295F0DF1D
:100586000895FF91EF910F93EE0FFF1F0591003035
:1005960031F010D00D30D1F70AE00CD0F7CF3196FC
:1005A600F695E7950F91EF93FF9308955F9BFECF26
:1005B6000CB108955D9BFECF0CB90895F502F602C5
:1005C600F802FA02FC02FE020003020304030B0314
:1005D6000E031103140317031C032103260333031D
:1005E600390344030895322D0895332D0895342D8B
:1005F6000895352D0895362D0895382D0895372DF3
:1006060008953B2F422D0DD23B7F10FF3460089595
:10061600342D432D0895362D452D0895372D482D1B
:100626000895392D4A2D0895632D542D34DF302F2A
:100636000895652D562D2FDF302F0895682D572DDF
:100646002ADF302F08956A2D592D25DF302F6A2D88
:10065600592D01E010E0500F611F1DDF402F089556
:10066600582F692F18DF0196302F0895582F692FBC
:1006760012DF302F0196582F692F0DDF0196402F7C
:100686000895582F692F07DF087340E0302F08952B
:100696006003610363036503670369036B036D030B
:1006A6006F03760379037C039B039E037F03840316
:1006B60089038E03A103A503AD030895232E089590
:1006C600332E0895432E0895532E0895632E0895CC
:1006D600832E0895732E0895242EB32F00E0F02E56
:1006E600B2FFF3940895342E432E0895542E632EAC
:1006F6000895842E732E0895632D542D032FF2DE54
:100706000895652D562D032FEDDE0895682D572D7E
:10071600032FE8DE08956A2D592D032FE3DE6A2D97
:10072600592D01E010E0500F611F042FDBDE089504
:10073600A42E932E0895942F832F089526D1832FC8
:10074600942F08953F934F93382F492F0DD19F91A2
:100756008F910895642F532F022DC4DE0895DA0376
:10076600DB03E903F803FD03020408040E0417047F
:100776002004300442045204670472047D04880491
:100786008F049C04A704AC04AF04B404B104C804E9
:10079600B704E204E704EC04F104F604FC040205E1
:1007A60007050C051005D904E004E10427050895A2
:1007B600B17001E0300F0FB7F32E01FBB6F937FD2C
:1007C600B06805FBB4F900FBB2F90895B170B260E8
:1007D60001E0301B0FB7F32E01FBB6F904FBB7F9A6
:1007E60005FBB4F900FBB2F9089501E010E0300F03
:1007F600411F089501E010E0301B410B0895BC7EB7
:10080600330F10F43160B1600895BC7E369510F454
:100816003068B16008958894B0FD089437950FB795
:10082600BC7E00FBB0F908958894B0FD0894331F90
:100836000FB7BC7E00FBB0F90895B0E0320D0FB7DC
:1008460001FBB6F904FB303809F4B06805FBB4F9CE
:1008560003FBB2F900FBB0F908958894B0FD089443
:10086600321D0FB7B0E001FBB6F937FDB06805FBE6
:10087600B4F903FBB2F900FBB0F9BD7F0895022D70
:10088600031B302F0FB701FBB6F904FBB7F905FBC5
:10089600B4F903FBB2F900FBB0F9B2600895022D7A
:1008A6008894B0FD0894030B302F0FB704FBB7F9FB
:1008B60005FBB4F903FBB2F900FBB0F930300FB712
:1008C60001FBB6F9B2600895B0E032210FB701FB23
:1008D600B6F904FBB7F905FBB4F9032F0895B0E0A8
:1008E60032290FB701FBB6F904FBB7F905FBB4F9DA
:1008F600032F0895B0E032250FB701FBB6F904FBCC
:10090600B7F905FBB4F9032F0895370D481D0FB746
:1009160000FBB0F9BD7F0895532F642F072DE2DD4C
:1009260001E010E0300F411F532F642F082DDADD50
:100936000895532F642FAFDD302F01E0500F00E0F4
:10094600601FA9DD402F0895532F642FA4DD302F9B
:1009560008957AD0032F0895B160089501E0B02775
:1009660008953095B261089501E010E0901AA10A49
:10097600592D6A2D042FB6DD01E010E0901AA10A68
:10098600592D6A2D032FAEDD0895592D6A2D83DD6D
:10099600302F01E010E0900EA11E592D6A2D7BDD4F
:1009A600402F01E010E0900EA11E0895082D842E20
:1009B600402F072D732E302F089508950895B6FF02
:1009C6000895A0E070E00895B6FD0895A0E070E0F7
:1009D6000895B0FF0895A0E070E00895B0FD089571
:1009E600A0E070E008951DD010FF0895A0E070E02B
:1009F600089517D010FD0895A0E070E00895B7FFA0
:100A06000895A0E070E00895B7FD0895A0E070E0B5
:100A16000895022D132FB6DB0895132FAEDB302F6A
:100A2600089511E0F0FC1395F1FC1395F2FC139573
:100A3600F3FC1395F4FC1395F5FC1395F6FC13954E
:100A4600F7FC1395117008959CDD496E76616C690B
:100A560064206F70636F646520402050433D000042
:100A6600092F8ADD082F88DDFFCF00003201C10182
:100A7600290D4204420851002114009C69412D00B1
:100A860029116304630871002118009C5201E101D9
:100A96004A0D8404840891002120009C6A412E009E
:100AA6004A11A504A508B100211C009C720112443C
:100AB6006B0DC604C608D1002150009C6B417249DB
:100AC6006B11E704E708F1002158009C920192029D
:100AD6008C0D0F060F0A11020054009C6C41324C1B
:100AE6008C11210421083100005C420043004400BF
:100AF6004500460047004F00410062006300640065
:100B06006500660067006F00610082008300840054
:100B16008500860087008F008100A200A300A40044
:100B2600A500A600A700AF00A100C200C300C40034
:100B3600C500C600C700CF00C100E200E300E40024
:100B4600E500E600E700EF00E1000202030204020E
:100B5600050206020702000001022200230024000B
:100B66002500260027002F002100222423242424E8
:100B76002524262427242F24212422282328242818
:100B86002528262827282F282128222C232C242CE8
:100B9600252C262C272C2F2C212C223023302430B8
:100BA6002530263027302F30213022342334243488
:100BB6002534263427342F342134223C233C243C4C
:100BC600253C263C273C2F3C213C22382338243820
:100BD6002538263827382F382138022C032C042CA8
:100BE600052C062C072C0F2C012C406A2061B269BB
:100BF600B201726A096431247302406E4002B26D1A
:100C0600009C726E72023128730240724061B271AA
:100C1600118872720A64312C73024076009CB27598
:100C2600318C7276009C31307302407A6061B27901
:100C36003092727A0B6431347302407EAB01B27D1E
:100C46004A91727E009C313C730240820061B281FF
:100C56000094728208643138730240868B01B28533
:0A0C660000987286009C112C7302A6
:00000001FF
